:100000000C9468020C94BA020C94BA020C94BA02D2
:100010000C94BA020C94BA020C94BA020C94BA0270
:100020000C94BA020C94BA020C94F41E0C94C61FE1
:100030000C94952D0C94BA020C94BA020C94BA024A
:100040000C94BA020C94BA020C94BA020C94BA0240
:100050000C94BA020C94AB0B0C94BA020C94BA0236
:100060000C94BA020C94BA020C94BA020C94BA0220
:100070000C94BA020C94BA020C94BA020C94BA0210
:100080000C94BA020C94BA020C94BA020C94BA0200
:100090000C94BA020C94BA020C94BA020C94BA02F0
:1000A0000C94BA020C94BA020C94BA023320552074
:1000B0004321552043219A20BD204321122125218F
:1000C000F723F723262426248424C224DC26DC26D6
:1000D000DB24DC26DC25DC25B026DC26DC26C72656
:1000E000808080800405060708090A0B0C0D0E0F9E
:1000F000101112131415161718191A1B1C1D1E1F88
:10010000202122232425262728292A2B2C2D2E2F77
:10011000303132333435363738393A3B3C3D3E3F67
:10012000404142434445464748494A4B4C4D4E4F57
:10013000505152535455565758595A5B5C5D5E5F47
:10014000606162636465666768696A6B6C6D6E6F37
:100150007071727380808080808080808080800356
:100160000201808080668075007476778080808050
:100170007677808080808080808080808080808092
:10018000808080808080808080808080808080806F
:10019000808080808080808080808080808080805F
:1001A000808080808080808080808080808080804F
:1001B000808080808080808080808080808080803F
:1001C00078797A7B7C7D7E7F808080808080808053
:1001D000808080808080808080808080808080801F
:1001E0000A00253031366200253032643A20000A98
:1001F000722F63203031323334353637383941424B
:10020000434445460A0073706565643A2025730AC5
:10021000007573625F73746174653A2025303258DB
:100220000A00686F73742E5461736B3A2025640A58
:10023000000D0A0020253032580073746174653A4D
:10024000202025303258202530325800696E6974DC
:100250003A20646F6E650A004368657272792062A5
:1002600075673A2069676E6F7265640D0A000D0A42
:1002700000202530325800696E7075742025643A6C
:10028000005B445D005B435D003C0355005300424E
:1002900000200074006F0020005500530042002031
:1002A000006B006500790062006F006100720064FD
:1002B00000200063006F006E00760065007200741D
:1002C000006500720000000E0374002E006D002E09
:1002D000006B002E000000040309040902740004EE
:1002E0000100A032090400000103010100092111ED
:1002F0000100012240000705810308000A090401EA
:10030000000103010200092111010001224D000733
:1003100005820308000A0904020001030000000925
:1003200021110100012236000705830308000A0994
:100330000403000203000000092111010001222230
:1003400000070584032000010705040320000112B3
:1003500001100100000008EDFE5B0014080102001E
:10036000010631FF0974A1010975150026FF0095EA
:1003700020750881020976150026FF009520750872
:100380009102C005010980A101850216810026B7EE
:10039000001A81002AB700751095018100C0050C74
:1003A0000901A1018503160100269C021A01002AF9
:1003B0009C02751095018100C005010902A1010987
:1003C00001A10005091901290515002501950575EB
:1003D000018102950175038101050109300931157B
:1003E00081257F95027508810609381581257F953D
:1003F0000175088106050C0A38021581257F9501D3
:1004000075088106C0C005010906A101050719E0AC
:1004100029E71500250195087501810295017508E8
:1004200081010508190129059505750191029501BC
:10043000750391010507190029FF150026FF009596
:100440000675088100C0636F6E73756D65723A2022
:10045000253034580A0073797374656D3A2025305D
:1004600034580A000A002530325820006B65796242
:100470006F6172643A20004C45443A20253032586E
:100480000A00290A002575002F002575005D280047
:10049000256400200025640020002564002000253C
:1004A00064007C0025303258006D6F7573656B6594
:1004B00079205B62746E7C782079207620685D28D4
:1004C0007265702F61636C293A205B00000AFF0A95
:1004D00011241FBECFEFDAE0DEBFCDBF04B603FEAE
:1004E00027C080918B0490918C04A0918D04B091D1
:1004F0008E048730904BA740B04BD1F410928B0400
:1005000010928C0410928D0410928E0414BE84B745
:10051000877F84BF0FB6F894A895809160008861AA
:1005200080936000109260000FBEE0E0F8E3099550
:1005300011E0A0E0B1E0E4E8F4E602C005900D921D
:10054000A839B107D9F724E0A8E9B1E001C01D92AC
:10055000AB38B207E1F712E0C8E6D2E004C0219759
:10056000FE010E942632C636D107C9F70E943B0A17
:100570000C9440320C940000FF93EF93E0919801AB
:10058000F0919901309709F00995EF91FF91089545
:10059000FC018591803011F0EFDFFBCF0895FF273C
:1005A000E0E230E247FF0CC0419597FF09C0EDE261
:1005B0006095709580959095611D711D811D911DAF
:1005C00027FF02C0219530E350E2AA27660F771F6C
:1005D000881F991FAA1FA41710F0A41B63955A9592
:1005E000A9F7AA3008F0A95FA05DAF93F395611554
:1005F00071058105910541F7ED3211F4EF93F39503
:10060000F21718F43F93F395FBCF8F91B5DFFA956E
:10061000E1F70895E991F9918591803021F08532D3
:1006200019F0AADFF9CF089520E0E89455915532EA
:10063000C1F3503311F4689455915A3348F4505330
:1006400090F3220F022E220F220F200D250FF4CF40
:100650000EF4219589919991533619F3533729F165
:10066000533559F1BC0188279927E8945C3621F469
:100670008991999168945591543639F446EF7EF0FA
:1006800077FF0DC08FEF9FEF0AC055374AE039F072
:10069000583540E121F0523642E009F00895FF93C9
:1006A000EF937DDFEF91FF91B7CFFF93EF93FC01C5
:1006B00081918030B9F360DFFBCFFF93EF9368DF68
:1006C000F1CFDF93CF93CDB7DEB72596A3DFCF91E0
:1006D000DF91089580E00895089580E0089581E015
:1006E0000895CF93DF93CDB7DEB728970FB6F89470
:1006F000DEBF0FBECDBF29833A834B835C836D83FE
:100700007E838F8398878091D202282B2093D202F8
:10071000FE013396AE01475F5F4F2191243088F090
:1007200080E090E0DC01AE52BD4F12963C911297F2
:10073000311103C012962C9304C0019686309105A6
:1007400089F7E417F50749F728960FB6F894DEBF46
:100750000FBECDBFDF91CF910895860F911D860FFB
:10076000911DFC015687458781E00895FC0187892A
:100770000895CF93DF93EC018C819D81DC01ED9195
:10078000FC910480F581E02D6E8109951F86188A01
:1007900081E08A8B1E821B8A1C8A1D8A1E8A1F8A00
:1007A00080E0DF91CF910895FC018681089581E07A
:1007B000633009F080E0089581E0613009F080E065
:1007C0000895860F911D860F911DFC0185859685E4
:1007D0000895EF92FF92CF93DF93DC01E7015296E9
:1007E0008C915297823049F11F966C931F975096C7
:1007F0004C9350979B8193709330F9F49A8197FFB3
:100800001CC09E8158962C915897291718F4589619
:100810009C935897E82FF0E09F01220F331FE20FBF
:10082000F31FEA0FFB1F9A819F7097839C8190872B
:1008300094E091878F5F52968C93DF91CF91FF90D8
:10084000EF900895EF92FF920F9302970E94E903B1
:100850000F91FF90EF9008950895DF92EF92FF922D
:100860000F931F93CF93DF93CDB7DEB762970FB689
:10087000F894DEBF0FBECDBFDC0157962C9122232A
:1008800081F07C010E94100BF701038914892589EE
:100890003689DC01CB01801B910BA20BB30BB7FF98
:1008A00002C0D12C39C0838590E09A8B898B8E0150
:1008B0000F5F1F4F9E012F5E3F4F428566818481EF
:1008C00095810E941514D82E811118C029893A8962
:1008D0002330310598F0D7011D968D919C911E977C
:1008E000009761F0DC01ED91FC910190F081E02D29
:1008F0008E010F5F1F4F40E0B70109950E94100B5A
:10090000F701208DDC01CB01820F911DA11DB11DCE
:10091000838B948BA58BB68B8D2D62960FB6F89436
:10092000DEBF0FBECDBFDF91CF911F910F91FF9022
:10093000EF90DF9008953F924F925F926F927F9277
:100940008F929F92AF92BF92CF92DF92EF92FF92DF
:100950000F931F93CF93DF93CDB7DEB7EC970FB60E
:10096000F894DEBF0FBECDBFDC0114968D909C9035
:10097000159716963C91311139C1522E342E462EC0
:100980005C01FC01108ED401ED91FC910190F0818D
:10099000E02D60E0C40109957C01009711F486ED1B
:1009A0002AC1FC01608071806114710409F420C1C6
:1009B0006501F7E0CF0ED11CDC011196DC92CE92DE
:1009C00014965C928E01065D1F4F28E030E040E0F7
:1009D00060E0F501848195810E94D8118CAF81116E
:1009E000F8C01AA5D7016D927C92D401ED91FC91CB
:1009F0000280F381E02D232D40E0642DC401099590
:100A0000F5018683882309F4F5C099A99087282FDA
:100A100040E060E0848195810E9483128CAFD40114
:100A2000ED91FC91D70114961C92882359F0048013
:100A3000F581E02DD50116966C91C4010995F5015B
:100A40001682D2C00190F081E02DD50116966C91EE
:100A5000C4010995FC01892B09F4A1CF912F133111
:100A600008F092E15482992369F0292F30E08E0139
:100A7000065D1F4F40E0F5016681848195810E94EB
:100A8000D8118CAF8CAD8111A7C0EBACF12C40E23A
:100A9000642E41E0742E2501F2E04F0E511C4E01F0
:100AA00081E1880E911CFE1449F17A8269825C8290
:100AB0004B821E86188A1F8619A21AA21BA219A68B
:100AC0009F828E82998688868D818B878A879D8674
:100AD0008C868E010F5F1F4F2F2D40E0D50116969B
:100AE0006C91169714968D919C9115970E942612E1
:100AF000F5018289823011F0F394D5CFD501529659
:100B00008C91823019F081ED8CAF66C0960142E085
:100B1000F5016681848195810E94120D8CAF68EE8B
:100B200073E080E090E00E94120BD5011F962C919B
:100B30001F9740E016966C91169714968D919C9194
:100B400015970E94F0138CAF811146C068EE73E0D8
:100B500080E090E00E94120B40E060E0C5010E943E
:100B6000E6158CAF811138C020E040E060E0C5019F
:100B70000E94BC158CAF86E291E09A838983AE0116
:100B80004F5F5F4F60E070E0C5010E944B1580E24F
:100B90008CAF8CAD8823C1F090E0959587958CAF94
:100BA000FE01FC966F01EE24E394F12C00E022E0BC
:100BB00040E060E0C5010E948E1569E170E080E0D0
:100BC00090E00E94120BE5CF91E0D50157969C93DF
:100BD00012C0F70171826082D501ED91FC91048011
:100BE000F581E02DC50109958CAD05C089ED03C0E7
:100BF00087ED01C084EDEC960FB6F894DEBF0FBE12
:100C0000CDBFDF91CF911F910F91FF90EF90DF90BB
:100C1000CF90BF90AF909F908F907F906F905F909C
:100C20004F903F9008950F931F93CF93DF93609160
:100C3000D2017091D301E091A101F091A201409104
:100C4000C6015091C7012091BA013091BB0180913A
:100C5000AE019091AF016E177F07B1F4E0919F0153
:100C6000F091A0014E175F0779F4E0919D01F0919A
:100C70009E012E173F0741F4E0919B01F0919C01EA
:100C80008E179F0709F49DC07093A2016093A10184
:100C90005093A00140939F0130939E0120939D01AA
:100CA00090939C0180939B01E2EDF2E088E0DF01EC
:100CB0001D928A95E9F72091CA013091CB014091AC
:100CC000CC015091CD016091CE017091CF01809106
:100CD000D0019091D1010E9471032091BE01309109
:100CE000BF014091C0015091C1016091C20170915A
:100CF000C3018091C4019091C5010E9471032091AC
:100D0000B2013091B3014091B4015091B5016091AD
:100D1000B6017091B7018091B8019091B9010E941C
:100D200071032091A6013091A7014091A801509133
:100D3000A9016091AA017091AB018091AC019091E1
:100D4000AD010E94710381E08093D1028091730410
:100D500080FF14C08091D3021F928F938091D202A2
:100D60001F928F938AE392E09F938F930E94610377
:100D70000F900F900F900F900F900F90C0E0D0E069
:100D800004E312E08091730480FF0EC0FE01EE5276
:100D9000FD4F82811F928F931F930F930E946103D7
:100DA0000F900F900F900F902196C630D10551F7FC
:100DB0008091730480FF07C081E392E00E94C80223
:100DC00002C01092D1020E94690BEC018AE592E008
:100DD0000E944C14CE010E94810B8536910580F053
:100DE0002091730420FF0CC09F938F9382E292E0C6
:100DF0009F938F930E9461030F900F900F900F901D
:100E0000C0919A018AE592E00E94EB0CC817B9F1F3
:100E10008AE592E00E94EB0C80939A019091730412
:100E200090FF0CC01F928F9381E192E09F938F936C
:100E30000E9461030F900F900F900F9080919A0184
:100E40008039E9F48091730480FF15C08091A3017B
:100E5000823019F088E191E002C083E191E09F9334
:100E60008F9386E092E09F938F930E9461030F908F
:100E70000F900F900F900E9460210E94D92281E074
:100E8000DF91CF911F910F910895482F50E0CA0133
:100E900024E0880F991F2A95E1F7805E9109089751
:100EA00030F48091D202882311F090E002C080E0FB
:100EB00090E0E4EDF2E0A1E0B0E036E03E0F2191F9
:100EC000243080F0622F62956F7070E046175707EC
:100ED00049F42F70BD0102C0660F771F2A95E2F713
:100EE000862B972B3E13EBCF0895EF92FF920F9333
:100EF0001F93CF93DF938FEE91E00E94C802C0E072
:100F0000D0E088EEE82E81E0F82E02EE11E0DF93CB
:100F1000CF93FF92EF920E9461038C2F0E944507AE
:100F20000E94632D9F938F931F930F930E946103E1
:100F300080EE91E00E94C80221968DB79EB7089678
:100F40000FB6F8949EBF0FBE8DBFC031D105F9F624
:100F5000DF91CF911F910F91FF90EF900895CF9265
:100F6000DF92EF92FF920F93CF93DF931F92CDB753
:100F7000DEB7898380913602882371F0CE01019615
:100F80006C01EE24E394F12C00E022E040E060E00C
:100F90008FE192E00E948E1580911D02882371F0EE
:100FA000CE0101966C01EE24E394F12C00E022E0E6
:100FB00040E060E086E092E00E948E15809104029D
:100FC000882371F0CE0101966C01EE24E394F12C9C
:100FD00000E022E040E060E08DEE91E00E948E159E
:100FE0008091EB01882371F0CE0101966C01EE2413
:100FF000E394F12C00E022E040E060E084ED91E039
:101000000E948E150F90DF91CF910F91FF90EF907E
:10101000DF90CF900895FC01758364838CE291E0AA
:10102000918380838AE491E093838283138A148A74
:10103000158A168A178A178288E080878CE3818751
:101040001286138684E0848781E0828B118A17865A
:101050001686158661157105B1F0DB01AA5ABF4FDE
:1010600080E090E02D913D91232B49F48B96880FE1
:10107000991FDB01A80FB91FED93FC93089501960A
:101080008031910579F708952E9A08952E988EBD96
:101090000DB407FEFDCF1EBC0DB407FEFDCF0E94B0
:1010A00044088EB508952E9882608EBD0DB407FE5B
:1010B000FDCF6EBD0DB407FEFDCF0C94440888EF44
:1010C0000E944608807C8034A1F018F4882301F146
:1010D0000895803819F0803CB9F0089588ED0E9499
:1010E000460881FD0BC069EC88ED0E94530882E040
:1010F0000CC088ED0E94460881FDF5CF6BEC88EDB1
:101100000E94530883E001C081E08093A301089509
:1011100061ED88ED0E9453081092A30108950F938A
:101120001F93CF93DF938C01269A0E944408219A43
:10113000229A2398209A80E58CBD81E08DBD259868
:1011400068E188E80E94530860E288E70E9453083B
:1011500060E088E70E945308C1E0D0E0209799F052
:1011600088E60E944608219680FFF8CF61EC88ED62
:101170000E94530860E680ED0E94530864E088EE08
:101180000E94530802C08FEF11C088EE0E944608EB
:1011900082FFFBCFC8010E945F0860E288EC0E94DA
:1011A000530861E080E80E94530880E0DF91CF910E
:1011B0001F910F9108958AE592E00E948F0888ECB4
:1011C00091E090932D0280932C028CEB91E0909310
:1011D00014028093130280EB91E09093FB018093C3
:1011E000FA0184EA91E09093E2018093E10108958D
:1011F000EF92FF920F931F93CF93DF93EC017B014C
:101200008A0188A1823029F128F4882341F08130B5
:1012100081F0C9C0833019F18430D9F1C4C082E0B3
:101220008C832D813E8138872F838A87898781E04F
:1012300088A3A801B701CE0107960E94D819811191
:1012400002C080E0B1C0ED81FE81808189A38181EF
:101250008AA3CE0142969E838D8383E088A38AA1D0
:10126000843059F018F4823049F00AC0853039F0E2
:10127000813231F489A1825002C01BA287E08C83A5
:101280008D819E8198878F838C818A87898784E06E
:1012900088A38AA1843081F0853091F1823009F0F1
:1012A00050C0A801B701CE0107960E94D819882323
:1012B00041F28D898CA372C0A801B701CE010796B7
:1012C0000E94D819882309F4BCCF8D89833009F096
:1012D00065C08E89813009F061C098A58F899923F6
:1012E00021F0882309F45AC003C0813009F056C0A8
:1012F00091E09BA39A899EA39B899FA38DA34EC037
:10130000A801B701CE0107960E94D819882309F4D5
:1013100098CF8BA1882309F441C08A819B810097D3
:10132000E9F1DC01ED91FC910190F081E02D7E016D
:10133000B0E1EB0EF11C0DA12FA14EA16CA10995FE
:101340002DC089A19D85992319F09130E9F021C024
:1013500090E002979F878E8781E08D8715C0F80106
:1013600020813181232BA9F001979F878E87F70178
:1013700080819181019691838083D8018D919C9188
:10138000119701978D939C938E859F85009739F7D0
:101390001D868E859F85892B09F053CFCE014096FF
:1013A0009E838D8318A281E0DF91CF911F910F91D1
:1013B000FF90EF9008950F931F93CF93DF9300D08A
:1013C00000D0CDB7DEB78C017C836B835A83498311
:1013D0002B813C81232B59F0AE014D5F5F4FBE0145
:1013E0006F5F7F4FC8010E94F8088111F1CF0F9005
:1013F0000F900F900F90DF91CF911F910F91089553
:101400008AE592E00E94BA0C6AE572E089E492E013
:101410000E946B186AE572E088E392E00E946B1804
:101420006AE572E08FE192E00E940B086AE572E0E3
:1014300086E092E00E940B086AE572E08DEE91E092
:101440000E940B086AE572E084ED91E00E940B08AF
:1014500080E591E09093C9018093C8019093BD010C
:101460008093BC019093B1018093B0019093A5014A
:101470008093A4010895569A5E9A809173048160C6
:1014800084608093730480E091E00E945B210E945D
:101490001C2284B7877F84BF0FB6F894A8958091EB
:1014A0006000886180936000109260000FBE90E041
:1014B00080E80FB6F89480936100909361000FBEAE
:1014C0000E94791E0E94D61E8091E2008460809363
:1014D000E20087E39AE10E94482D7894809173049A
:1014E00080FF04C08CE492E00E94C8020E94202287
:1014F000FDCFAF92BF92CF92DF92EF92FF920F9308
:101500001F93CF93DF937C01B22E8091730480FFF1
:1015100014C0DB01ED91FC910084F185E02DCB013D
:1015200009951F928F9387E792E09F938F930E9474
:1015300061030F900F900F900F90A02EC02FD12F0E
:1015400081E7C82E82E0D82E809173049C2F9A19CF
:101550009B1578F480FF0BC088811F928F93DF92D8
:10156000CF920E9461030F900F900F900F902196E1
:10157000EBCF80FF04C08EE692E00E94C802D80143
:1015800011968C91813091F48091730480FF1BC07F
:1015900088E592E0DF91CF911F910F91FF90EF903E
:1015A000DF90CF90BF90AF900C94C802D7011296F5
:1015B00088E0F80101900D928A95E1F70E94100BE6
:1015C000F70173876287DF91CF911F910F91FF9091
:1015D000EF90DF90CF90BF90AF900895089580E096
:1015E00090E008958FEF9FEF08958FEF9FEF08959C
:1015F0000895862F0E94371A81E090E00895EAED61
:10160000F2E01382128288EE93E0A0E0B0E08483DF
:101610009583A683B78386E591E0918380830895BF
:101620000C94750B8F929F92AF92BF92CF92DF92E4
:10163000EF92FF920E94E2304B015C0120E030E02B
:101640004AE755E40E9499316B017C0120E030E0CB
:1016500040E85FE30E94A73087FD24C020E03FEF11
:101660004FE757E4C701B6010E9494311816ACF455
:1016700020E030E040E251E4C501B4010E9499311C
:101680000E94B33020E931E06115710581F0C90194
:101690000197F1F761507109F7CFC701B6010E94B8
:1016A000B33002C061E070E0CB010197F1F7FF9029
:1016B000EF90DF90CF90BF90AF909F908F90089564
:1016C00082E084BD93E095BD9AEF97BD80936E0054
:1016D00008952FB7F8948091E8029091E902A091C3
:1016E000EA02B091EB022FBF08952FB7F8946091F2
:1016F000E8027091E9028091EA029091EB022FBF1B
:101700000895CF92DF92EF92FF920F931F932FB71E
:10171000F8944091E8025091E9026091EA027091D8
:10172000EB022FBF6A017B01EE24FF248C0120E035
:1017300030E0C016D106E206F30610F4415051091C
:101740009A01281B390BC9011F910F91FF90EF904F
:10175000DF90CF9008951F920F920FB60F92112431
:101760008F939F93AF93BF938091E8029091E9028A
:10177000A091EA02B091EB020196A11DB11D8093E8
:10178000E8029093E902A093EA02B093EB02BF91C2
:10179000AF919F918F910F900FBE0F901F90189552
:1017A000CF93DF93FC01862F807809F051C0283059
:1017B00008F04FC0442321F09581973009F449C0C7
:1017C000EF012D96A0E0B0E011969881911103C031
:1017D000662331F021C02596AF30B105A9F739C095
:1017E00085E08A9FE0018B9FD00D1124CE0FDF1F73
:1017F000442331F081E4888785818F5F858302C02F
:1018000081E0888725E02A9FC0012B9F900D11243D
:10181000E80FF91F80851DC06770660F660F660FA1
:10182000442341F0606485818F5F85838770687F82
:10183000682B03C02770687B622B25E02A9FC001BC
:101840002B9F900D1124E80FF91F6087862F01C090
:1018500080E0DF91CF910895DF92EF92FF920F9396
:101860001F93CF93DF93EC01E62EF12C85E0689F68
:10187000B0011124FE01E60FF71F8085182F1770A5
:1018800086FF21C001E085E0D82E8FEF800F8F30DA
:1018900008F001E0FE01D09EE00DF11D11248085CD
:1018A0008695869586958770811305C0602FCE0139
:1018B0000E942C0CEACF0F5F003161F78D818113FC
:1018C00002C011501D8385E08E9DF0018F9DF00DAB
:1018D0001124EC0FFD1F108681E08187128622966D
:1018E000D783C683DF91CF911F910F91FF90EF9027
:1018F000DF900895611102C006960895FC013D969F
:1019000021E03081361307C035E0239F800D911D03
:101910001124069608952F5F3596203191F780E0C7
:1019200090E00895FC016134C1F43F969C01265A71
:101930003F4F61E0AC014E5F5F4FDF0112971C9299
:1019400011966C93108213974D935C933596E21722
:10195000F30799F7FC01158208953D9621E0308147
:10196000361303C0622F0C942C0C2F5F3596203158
:10197000B1F70895CF93DF93FC0188E691E091835E
:1019800080831582108681E081871286CF010296BE
:1019900097838683128228E023832CE32483DF014C
:1019A0001F969F01265A3F4F41E0ED012297188272
:1019B000219648831C922397998388831596A217B2
:1019C000B30799F7EA58FF4F108281E18093F00244
:1019D000DF91CF9108958091F0020895CF93DF9326
:1019E0001F92CDB7DEB749830E947A0C49810097D8
:1019F00089F0DC01ED91FC911197309759F0139625
:101A00009C9180E0891731F02081241731F03396C2
:101A10008F5FF8CF80E090E001C0CF010F90DF91A1
:101A2000CF9108950F931F93CF93DF932115310525
:101A300071F0E901042F162F0E947A0CFC01892B0A
:101A400041F01283D183C083038380E003C088ED1B
:101A500001C086EDDF91CF911F910F910895CF9234
:101A6000DF92FF920F931F93CF93DF93662381F151
:101A7000F62E8C016C0186E5C80ED11CC0E0D0E0CA
:101A8000D6018D919D916D010097F1F0DC01ED91F2
:101A9000FC910084F185E02D09958F1115C0AB965E
:101AA000CC0FDD1FC00FD11F88819981DC01ED9122
:101AB000FC910480F581E02DDF91CF911F910F9172
:101AC000FF90DF90CF9009942196C031D105C1F6E7
:101AD00080E0DF91CF911F910F91FF90DF90CF9029
:101AE00008952E980895CF93DF931F92CDB7DEB758
:101AF00089830E94710D89818EBD0DB407FEFDCFD3
:101B00001EBC0DB407FEFDCF0E9444088EB50F9099
:101B1000DF91CF910895CF93DF9300D0CDB7DEB79B
:101B20006A8389830E94710D898182608EBD6A817A
:101B30000DB407FEFDCF6EBD0DB407FEFDCF0F90B7
:101B40000F90DF91CF910C9444088F929F92AF92A7
:101B5000BF92DF92EF92FF920F931F93CF93DF9389
:101B60001F92CDB7DEB74C01D62E590149830E9492
:101B70007A0C7C014981009709F440C0FC01808106
:101B80009181892BE9F16D2DC4010E94EE0CF501C4
:101B9000918380830097B1F1FC01228126952695DF
:101BA00030E02031310514F02FE030E081E090E0AA
:101BB000A0E0B0E004C0880F991FAA1FBB1F2A95A0
:101BC000D2F70197F801918380836D2D80EE0E94FA
:101BD0008B0D88ED0E94730D682FF7018481882397
:101BE00039F0F401EA58FF4F80818260682B01C010
:101BF000697F88ED0E948B0D80E005C086ED03C0F3
:101C000087ED01C08BED0F90DF91CF911F910F9168
:101C1000FF90EF90DF90BF90AF909F908F900895CE
:101C20008F929F92AF92BF92CF92DF92EF92FF92EC
:101C30000F931F93CF93DF93862E942E59010E940A
:101C4000100B6B017C0128E8C20E23E1D21EE11CBF
:101C5000F11C00E010E0D0E0C0E098280E94100BDA
:101C6000DC01CB018C199D09AE09BF09B7FF2DC05E
:101C7000692D80EF0E948B0D0E94100BDC01CB01BF
:101C80008C199D09AE09BF09B7FF09C088EC0E94F5
:101C9000730D87FFF1CF60E888EC0E948B0D88EF11
:101CA0000E94730DC82FCF70C43019F0CE3051F0A0
:101CB0000CC00F5F1F4FA114B10481F20A151B0560
:101CC00069F603C0DF5FD33049F68C2FDF91CF91E7
:101CD0001F910F91FF90EF90DF90CF90BF90AF904A
:101CE0009F908F9008959F92AF92BF92CF92DF9274
:101CF000EF92FF920F931F93CF93DF937C01C42F3A
:101D0000122F992493946C01C60ED11CC60ED11CBF
:101D100086E5C80ED11CA42EB12CABE2AA0EB11CD4
:101D2000AA0CBB1CAE0CBF1CF60180819181DC01AA
:101D3000ED91FC910280F381E02D202F412F6C2F3B
:101D40000995803EC9F4C1110BC061E088EE0E9484
:101D50008B0D66E670E080E090E00E94120B16C0EA
:101D6000F50180819181DC01ED91FC910284F38584
:101D7000E02D612F09950AC08D3031F49FEF990D48
:101D8000933008F040C016C081113DC0F60180813B
:101D90009181DC01ED91FC910190F081E02D202FEB
:101DA000412F6C2F0995D82F8D3061F48FEF890D5D
:101DB000833050F464E670E080E090E00E94120B03
:101DC0009394B2CF8823F1F0C1110BC061E088EE8B
:101DD0000E948B0D66E670E080E090E00E94120B9E
:101DE00011C0EC2FF0E0BB96EE0FFF1FEE0DFF1DB4
:101DF00080819181DC01ED91FC910284F385E02DDD
:101E0000612F09958D2FDF91CF911F910F91FF9039
:101E1000EF90DF90CF90BF90AF909F9008950F9379
:101E20001F93CF93DF9300D0CDB7DEB78A016A83CB
:101E300089830E94710D898182608EBDF8016A815B
:101E4000862F882339F00DB407FEFDCF91919EBDFA
:101E50008150F7CF060F111D0DB407FEFDCF0E9474
:101E60004408C8010F900F90DF91CF911F910F91FF
:101E700008952F923F924F925F926F927F928F922E
:101E80009F92AF92BF92CF92DF92EF92FF920F9309
:101E90001F93CF93DF9300D000D01F92CDB7DEB752
:101EA0007D836C835A016901FB0121808FEF820DD4
:101EB000803408F075C00E94100B2B013C01F8E83B
:101EC0004F0EF3E15F1E611C711CEC81FD8182816C
:101ED00080FD02C060E401C060E888EE0E948B0DC6
:101EE00020E0312CC114D10409F44AC076012C142D
:101EF0003D0408F47101EA82A8016E2D80E10E9480
:101F00000F0F6E2D88E30E948B0DEC81FD816081A7
:101F1000606280EF0E948B0D88EC0E94730D87FF3A
:101F2000FBCF60E888EC0E948B0D88EF0E94730D58
:101F3000282F2F70812C912C1982222361F02B8362
:101F40000E94100BDC01CB0184199509A609B70981
:101F50002B81B7FD05C0CE18DF080E0D1F1DC2CFA7
:101F6000263001F12E3009F456C0243049F4FFEF39
:101F70008F1A9F0AA114B10459F18A149B0441F5E8
:101F800088EF2B830E94730D85FB882780F9EC81F5
:101F9000FD81928180FB90F992832B81822F41C039
:101FA0008AED3FC088EF0E94730D85FB882780F97A
:101FB00091E08927EC81FD81928180FB90F99283E9
:101FC00090FD02C060E401C060E888EE0E948B0DC5
:101FD00060E088E30E948B0DF801608180E10E943F
:101FE0008B0D6A8188E30E948B0DEC81FD816081FD
:101FF000606280EF0E948B0D88EC0E94730D87FF5A
:10200000FBCF60E888EC0E948B0D88EF0E94730D77
:10201000282F2F7092CF89818F5F89838330C1F6FB
:10202000AFCF0F900F900F900F900F90DF91CF9147
:102030001F910F91FF90EF90DF90CF90BF90AF90E6
:102040009F908F907F906F905F904F903F902F90D8
:1020500008952F923F924F925F926F927F928F924C
:102060009F92AF92BF92CF92DF92EF92FF920F9327
:102070001F93CF93DF9300D000D01F92CDB7DEB770
:102080005C017D836C834A017901F901C080D180B4
:10209000FB014180F90111821082FB01828181FDE7
:1020A00002C060E101C060E288EE0E948B0D3C2C12
:1020B0009401EC81FD81408160E0C5010E94100E19
:1020C000582EF6E08F1316C088EF0E94730D82958C
:1020D000817091E08927EC81FD81928180FB91F9EB
:1020E000928391FD02C060E101C060E288EE0E942F
:1020F0008B0DDECF81115BC088EC0E94730D82FFD7
:1021000054C080E30E94730D282E282F30E0C216A1
:10211000D30608F4232CF70120813181622C712C25
:10212000A601421B530B57FF02C040E050E0930151
:10213000461557050CF49A0129833A832B830E9494
:10214000710DF8E0FEBD8B813A8129810DB407FE47
:10215000FDCFF801882341F01EBC81500DB407FE6D
:10216000FDCF4EB54193F6CF020F131F0E944408D6
:1021700064E088EC0E948B0DF70120813181620EB2
:10218000731E71826082241420F06C147D0408F4A4
:102190008FCF88EF0E94730D82958170EC81FD8155
:1021A000928180FB91F9928302C080EF582E852D99
:1021B0000F900F900F900F900F90DF91CF911F9184
:1021C0000F91FF90EF90DF90CF90BF90AF909F90D6
:1021D0008F907F906F905F904F903F902F900895D9
:1021E0002F923F924F925F926F927F928F929F9227
:1021F000AF92BF92CF92DF92EF92FF920F931F9315
:10220000CF93DF93CDB7DEB762970FB6F894DEBFFA
:102210000FBECDBF3C01542ED22E402E5E2D2FA0DE
:1022200038A4E9A4FAA4188A1F861E861D868E018A
:10223000035F1F4F9E01215F3F4F598B0E94A50DE9
:10224000598981119CC0D9824A825B83CC82BE822B
:10225000AD8298868F82AE014F5F5F4F68E080E26B
:102260000E940F0F2D853E85452D60E1C3010E9420
:10227000100E182F81117FC0BD2CBB1CBB24BB1CB2
:10228000E114F10409F46AC0EF85F8898281BB206A
:1022900009F455C0826082836401AA24A394C11406
:1022A000D10409F449C03C862B864D855E856F8537
:1022B000788987019E01255F3F4FC3010E94291045
:1022C000182F8630B1F42F85388988EF298B3A8B07
:1022D0000E94730D85FB882780F98A2529893A8910
:1022E000D90112969C91129780FB91F912969C93BA
:1022F000D6CF811140C0EBA5FCA53097A1F001908D
:10230000F081E02D0190F081E02DC4018C199D0930
:102310009A8789876B857C859E01275F3F4FA70140
:102320008BA59CA509958B859C85C81AD90A821511
:10233000930508F0B4CF12C011111DC014C0816004
:1023400082834D855E8587019101BF01C3010E9493
:10235000390F811114C02D853E850FC02D853E8516
:10236000B11003C00AC02D853E8560EA452DC3012A
:102370000E94100E04C0812F02C060E8F7CF629661
:102380000FB6F894DEBF0FBECDBFDF91CF911F9186
:102390000F91FF90EF90DF90CF90BF90AF909F9004
:1023A0008F907F906F905F904F903F902F90089507
:1023B0008F929F92AF92BF92CF92EF920F931F9303
:1023C0001F921F921F930F933F932F934901A12CAC
:1023D000B12CCC24C394E12C06E020E80E94F0103C
:1023E0000F900F900F900F900F900F901F910F91E3
:1023F000EF90CF90BF90AF909F908F9008958F9265
:102400009F92AF92BF92CF92EF92FF920F931F9243
:102410001F92FF92EF923F932F934901A12CB12C71
:1024200022E0C22EE02E06E020E80E94F0100F907D
:102430000F900F900F900F900F900F91FF90EF90D3
:10244000CF90BF90AF909F908F9008954F925F92E2
:102450006F927F928F929F92AF92BF92CF92DF92B4
:10246000EF92FF920F931F93CF93DF93CDB7DEB719
:10247000C054D1090FB6F894DEBF0FBECDBF3C01EA
:10248000D62E542E422EC02ECE0101965C017C0128
:10249000022F29E030E0C3010E94FF1181111BC00F
:1024A0008B809C801F93CF92BF92AF921F9280E44B
:1024B0008F93A12CB12C82E0C82EE42C06E020E8FA
:1024C000452D6D2DC3010E94F0100F900F900F90BD
:1024D0000F900F900F90C05CDF4F0FB6F894DEBFE7
:1024E0000FBECDBFDF91CF911F910F91FF90EF9065
:1024F000DF90CF90BF90AF909F908F907F906F9024
:102500005F904F9008958F929F92AF92BF92CF921B
:10251000EF920F93CF931F921F921F921F921F92C1
:102520001F92812C912CA12CB12CC12CE22E05E004
:1025300020E00E94F010C82F6CE271E080E090E093
:102540000E94120B0F900F900F900F900F900F9012
:102550008C2FCF910F91EF90CF90BF90AF909F9025
:102560008F9008950F931F93CF93DF938A3F3FEF90
:10257000930711F486ED2DC0DC011696ED91FC91C8
:102580001797EF2B09F1122F242FEC011A8740E047
:102590000E94D00B082F8823C9F0682FCE010E941B
:1025A0007A0C009739F3FC011483202F40E060E09F
:1025B000CE010E948312182F882351F0602FCE0184
:1025C0000E94920C812F05C087ED03C084ED01C0ED
:1025D00080E0DF91CF911F910F9108952F923F924C
:1025E0004F925F926F927F928F929F92AF92BF9223
:1025F000CF92DF92EF92FF920F931F93CF93DF93CF
:10260000CDB7DEB766970FB6F894DEBF0FBECDBF6D
:102610001B8A38E03C8B3CE33D8B8A3F3FEF9307BE
:1026200009F4ADC0B22E342EA62E7C01DC01169624
:10263000CD90DC901797CE01439617969C938E937E
:1026400016971A962C938E010F5F1F4F22E130E0F0
:1026500040E060E0C7010E94D811F701D782C6822E
:102660008111A5C069847A844B845C843D813E8B52
:102670002E80670186E5C80ED11C460110E0D4010A
:102680008D919C91009789F1DC01ED91FC91008482
:10269000F185E02D0995811128C0F4018081918197
:1026A000DC01ED91FC910088F189E02D622D099506
:1026B0008823D9F0F40180819181DC01ED91FC91B6
:1026C0000484F585E02DA201B3010995811159C05B
:1026D000F40180819181DC01ED91FC910684F78504
:1026E000E02D6E89099581114CC01F5FB2E08B0E01
:1026F000911C103121F610E0F60180819181009744
:1027000089F1DC01ED91FC910084F185E02D0995C2
:10271000811128C0F60180819181DC01ED91FC914D
:102720000088F189E02D622D09958823A9F1F60131
:1027300080819181DC01ED91FC910484F585E02D8F
:10274000A201B301099581110DC0F601808191812B
:10275000DC01ED91FC910684F785E02D6E890995E9
:102760008823D1F01F5FB2E0CB0ED11C103121F6CF
:102770002B2D432D6A2DC7010E94B21218C086ED81
:1027800016C00B2D232D4A2D612FC7010E94730EF9
:10279000813D09F4AACF0BC00B2D232D4A2D612FAB
:1027A000C7010E94730E982F977F913DD9F26696CC
:1027B0000FB6F894DEBF0FBECDBFDF91CF911F9152
:1027C0000F91FF90EF90DF90CF90BF90AF909F90D0
:1027D0008F907F906F905F904F903F902F900895D3
:1027E0008F929F92AF92BF92CF92EF920F931F92D0
:1027F0001F921F921F921F921F92812C912CA12C2D
:10280000B12CC12CE22E09E020E00E94F0100F90C4
:102810000F900F900F900F900F900F91EF90CF901F
:10282000BF90AF909F908F900895AF92BF92CF923C
:10283000DF92EF92FF920F931F93CF93DF9300D01D
:1028400000D0CDB7DEB77C01690158011C821B8224
:102850001A8219828E010F5F1F4F9E012D5F3F4F1D
:102860000E94A50D811109C049815A816B817C812B
:1028700085019601C7010E9429100F900F900F90BB
:102880000F90DF91CF911F910F91FF90EF90DF900C
:10289000CF90BF90AF900895AF92BF92CF92DF924A
:1028A000EF92FF920F931F93CF938C011D990EC04F
:1028B00088EC0E94730D85FF05C0C8010E945F0867
:1028C00060E201C060E088EC0E948B0D8091A30162
:1028D000813039F040F0823079F0833039F5C1E051
:1028E0000CC083E106C08091F002807F8031F1F05E
:1028F00081E18093F0021AC0C0E08091F002807FF5
:102900008031A9F40E94100BDC01CB0188539F4F4A
:10291000AF4FBF4F8093EC029093ED02A093EE0275
:10292000B093EF0280E28093F00201C0C0E0780132
:1029300086E5E80EF11C6801A6E7CA0ED11C570116
:10294000F501819191915F01009739F0DC01ED91E2
:10295000FC910680F781E02D0995AC14BD0481F748
:102960009091F002903409F43FC050F4903221F17C
:102970009033A1F1913109F084C0F60110820AC0B0
:10298000913509F458C0903809F46AC0903509F0BF
:1029900078C039C0D7018D919D917D01009739F0A4
:1029A000DC01ED91FC910480F581E02D0995EC149A
:1029B000FD0481F782E163C00E94100B0091EC02DC
:1029C0001091ED022091EE023091EF02DC01CB017B
:1029D000801B910BA20BB30BB7FD53C061E088EED7
:1029E0000E948B0D80E44BC088EE0E94730D80FD29
:1029F00048C088ED0E94730D682F686088ED0E94C2
:102A00008B0D80E53CC088EC0E94730D86FF39C0B9
:102A100081E58093F0020E94100BDC01CB0144960B
:102A2000A11DB11D8093EC029093ED02A093EE02E4
:102A3000B093EF0226C00E94100BC090EC02D09021
:102A4000ED02E090EE02F090EF02DC01CB018C1978
:102A50009D09AE09BF09B7FD14C080E88093F0025C
:102A60002C2F40E060E0C8010E94EE12882331F074
:102A7000823D39F08093F10280EA01C080E98093C1
:102A8000F002CF911F910F91FF90EF90DF90CF90C8
:102A9000BF90AF9008958F929F92AF92BF92CF92C6
:102AA000EF920F93CF93DF93CDB7DEB7C054D10928
:102AB0000FB6F894DEBF0FBECDBF5F934F939E015C
:102AC0002F5F3F4F3F932F931F9220E42F9320E8D7
:102AD000822E912C5B0132E2C32EE12C06E021E82C
:102AE00040E0FC016681848195810E94F0100F9086
:102AF0000F900F900F900F900F90C05CDF4F0FB6AC
:102B0000F894DEBF0FBECDBFDF91CF910F91EF9054
:102B1000CF90BF90AF909F908F9008958F929F928B
:102B2000AF92BF92CF92DF92EF92FF920F938E2CD3
:102B3000A42EB12C1F921F92DF92CF92FF92EF92A0
:102B40009F2CC22EE02E09E021E2462FFC01668177
:102B5000848195810E94F0100F900F900F900F903C
:102B60000F900F900F91FF90EF90DF90CF90BF905C
:102B7000AF909F908F9008958F929F92AF92BF9247
:102B8000CF92EF920F93A62EB12C1F921F921F92FD
:102B90001F921F921F92812C912CC22EE42E0AE0CC
:102BA00021E240E0FC016681848195810E94F01061
:102BB0000F900F900F900F900F900F900F91EF903C
:102BC000CF90BF90AF909F908F9008958F929F92DB
:102BD000AF92BF92CF92EF920F93A62EB12C1F927D
:102BE0001F921F921F921F921F92812C912CC12C19
:102BF000E42E0BE021E240E0FC01668184819581B6
:102C00000E94F0100F900F900F900F900F900F9068
:102C10000F91EF90CF90BF90AF909F908F900895BD
:102C2000FC018285089581E0693009F080E0089513
:102C3000CF93DF93EC018A819B81DC01ED91FC91C4
:102C40000480F581E02D6A8509958A85813439F4FF
:102C5000EA81FB81EA58FF4F8081846080831A8675
:102C60001B861C861D861E861F86188A80E0DF91C3
:102C7000CF9108958F929F92AF92BF92CF92EF9291
:102C80000F93A42EB12CB22A1F921F921F921F9253
:102C90001F921F92812C912CC12CE62E01E023E281
:102CA00040E0FC016285828193810E94F0100F90C8
:102CB0000F900F900F900F900F900F91EF90CF907B
:102CC000BF90AF909F908F9008958F929F92AF92F8
:102CD000BF92CF92EF920F93A62EB12C1F921F920C
:102CE0003F932F935F934F934A01C12CE12C00E057
:102CF00023EA40E0FC016285828193810E94F0100A
:102D00000F900F900F900F900F900F900F91EF90EA
:102D1000CF90BF90AF909F908F9008958F929F9289
:102D2000AF92BF92CF92EF920F93A42EB12CB22A02
:102D30001F921F921F921F921F921F92812C912C03
:102D4000C12CE62E03E023E240E0FC016285828193
:102D500093810E94F0100F900F900F900F900F90A2
:102D60000F900F91EF90CF90BF90AF909F908F906A
:102D700008952F923F924F925F926F927F928F921F
:102D80009F92AF92BF92CF92DF92EF92FF920F93FA
:102D90001F93CF93DF93CDB7DEB7E8970FB6F894C4
:102DA000DEBF0FBECDBFDC011296ED90FC901397F5
:102DB0001A963C91311104C1122F242E362E3C015B
:102DC000D701ED91FC910190F081E02D60E0C70109
:102DD00009956C01009709F4F5C0FC01A080B18051
:102DE000A114B10409F4F0C04301F4E08F0E911C6A
:102DF000DC0111969C928E9214961C93FE013196E2
:102E00002F018F0128E030E040E060E0D30112960E
:102E10008D919C9113970E94D811F6011482811113
:102E2000D9C009818D81893009F0D0C0D701ED91D9
:102E3000FC910280F381E02D222D41E0632DC7013A
:102E40000995F3018287882309F4C2C09885958388
:102E5000282F40E060E0828193810E948312182F26
:102E6000882389F0D601AD92BC92D701ED91FC91F7
:102E70000480F581E02DD3011A966C91C701099564
:102E8000F3011286ABC0202F013208F020E2D601F8
:102E9000AD92BC9221110BC0940142E0F301628516
:102EA000828193810E94120D811197C010C030E081
:102EB000820140E0D3011A966C911A9712968D9177
:102EC0009C9113970E94D811811187C0E5CF1F9262
:102ED0001F925F924F921F9288E08F9388E0882E16
:102EE000912CA12CB12C99E2C92EE12C06E020EA0C
:102EF00040E0F3016285828193810E94F010182FD7
:102F00000F900F900F900F900F900F90811166C04F
:102F10008B81D3011B968C931B97720100E028E0F4
:102F200030E040E01A966C911A9712968D919C9120
:102F300013970E94FF11811150C02B813C8140E00A
:102F4000F3016285828193810E94FF11811145C046
:102F5000298130E0CE0181967C0140E0D3011A96B0
:102F60006C911A9712968D919C9113970E94FF1164
:102F7000811133C02E8140E0F3016285828193810B
:102F80000E94F013811129C001E0D3011B968C919E
:102F90001B97801740F020E0402F68E0C3010E949B
:102FA0008E160F5FF2CF1296ED91FC911397EA58AF
:102FB000FF4F80818460808381E050968C930EC0A7
:102FC00019ED0CC016ED0AC017ED08C011ED06C0D2
:102FD00014ED04C0F601B182A082182F812FE8966B
:102FE0000FB6F894DEBF0FBECDBFDF91CF911F911A
:102FF0000F91FF90EF90DF90CF90BF90AF909F9098
:103000008F907F906F905F904F903F902F9008959A
:10301000CF92DF92FF920F931F93CF93DF9300D055
:1030200000D0CDB7DEB78C01F62E19821A821B8232
:103030001C8220E0462F61E10E943A1620E04F2DCD
:1030400060E1C8010E943A1620E04F2D64E0C801FB
:103050000E948E1683E0C82ED12C9E012F5F3F4F19
:1030600044E050E06F2DC8010E9465168823F1F0FE
:1030700020E04F2D64E1C8010E943A1620E04F2D58
:1030800060E1C8010E943A1664E170E080E090E0DF
:103090000E94120B0F900F900F900F90DF91CF9125
:1030A0001F910F91FF90DF90CF90089589819A81B1
:1030B000AB81BC819D7F83309140A041B105C1F2BD
:1030C00064E670E080E090E00E94120B81E0C81A94
:1030D000D10819F6CDCFFC0182E791E0918380837E
:1030E0007383628312861386148615861686178666
:1030F000108A148288E085839CE3968391E097830D
:10310000808784E0818761157105B1F0DB01AA5ADF
:10311000BF4F80E090E02D913D91232B49F48B9699
:10312000880F991FDB01A80FB91FED93FC93089539
:1031300001968031910579F70895EF92FF920F93F0
:103140001F93CF938C01C62F7A01FA018081918160
:10315000A281B3818130F3E09F07F1E0AF07B105B1
:10316000D1F060F48115E1E09E07AE07B10571F181
:1031700081309140A140B10571F064C0833021E0FD
:10318000920720E1A207B105E1F183309340A0410D
:10319000B105B9F157C08091F202811153C020E00E
:1031A0004C2F61E1C8010E943A1620E04C2F60E1EB
:1031B000C8010E943A1620E04C2F64E0C8010E942A
:1031C0008E1681E08093F20281EB3DC020E0462F15
:1031D00061E1C8010E943A1620E04C2F60E1C8016D
:1031E0000E943A161092F202F80162856770C77069
:1031F000660F660F660F6C2B828193810E942F0DE4
:1032000021C020E04C2F64E1C8010E943A1620E062
:103210004C2F60E1C8010E943A1664E170E080E042
:1032200090E00E94120BF8016285F701218126953A
:10323000217067704C2FF801828193810E94EE12F9
:103240001092F20280E0CF911F910F91FF90EF90CA
:103250000895EF92FF920F931F93CF93DF93CDB713
:10326000DEB72E970FB6F894DEBF0FBECDBF7C0140
:1032700081E090E09E878D878E010F5F1F4F9E013A
:10328000235F3F4F41E0F7016285828193810E9475
:103290001514811151C002E011E089818023D1F021
:1032A00019861A861B861C869E01275F3F4F44E0C5
:1032B00050E0612FC7010E94651681110BC0AE015D
:1032C000475F5F4F612FC7010E949D18813B99F1B5
:1032D000811132C0000F1F5F1830F9F611E0F701BD
:1032E0008385811740F119861A861B861C869E01EC
:1032F000275F3F4F44E050E0612FC7010E946516F1
:10330000811117C089859A858770917081309140AD
:1033100081F48B859C8581609C878B87AE01475F9C
:103320005F4F612FC7010E949D18813B21F08111E1
:1033300003C01F5FD4CF80E02E960FB6F894DEBF97
:103340000FBECDBFDF91CF911F910F91FF90EF90F6
:1033500008950F931F93CF93DF93FC0120892111D0
:1033600002C080E020C0EC010E94100B0C851D857E
:103370002E853F85DC01CB01801B910BA20BB30B8B
:10338000B7FDEFCFCE010E942919182F0E94100B14
:10339000DC01CB018C599F4FAF4FBF4F8C879D876E
:1033A000AE87BF87812FDF91CF911F910F91089535
:1033B000CF93DF93FC01EA0180819181892B19F57C
:1033C00080E027C028813981232BD1F3DB012D91A7
:1033D0003C91D9019C91A381B0E0A81BB109208147
:1033E0003181A20FB31F9C93828181508283888197
:1033F0009981019799838883DB018D919C91119725
:1034000001968D939C9382818111DCCF838182838D
:1034100081E0DF91CF910895CF92DF92EF92FF92FA
:103420000F931F93CF93DF936C01EB017B01E40EAD
:10343000F51E00E010E0CE15DF0561F06991D601C0
:10344000ED91FC910190F081E02DC6010995080FE6
:10345000191FF1CFC801DF91CF911F910F91FF90FC
:10346000EF90DF90CF9008958091FF0208959FB76D
:10347000F8941092F6029FBF90918204943009F064
:1034800057C09091E9009F703091EC00232F21707C
:1034900030FD20E8922B24E02093E9002091EB00FE
:1034A00020FF43C02091EE0027FF3FC02091F30290
:1034B000222321F02091E80025FF37C01092F3026B
:1034C00026E03091E80035FD15C03091820434309B
:1034D00061F53091EB0035FD28C0215021F481E0E9
:1034E0008093F30222C0EFE9FFE03197F1F700C0CB
:1034F0000000E7CF8093F1008091E80085FD0AC0CD
:103500008091E80080FFFCCF8091E8008E77809367
:10351000E80006C08FB7F89421E02093F6028FBF31
:103520009F709093E90080E008959F709093E90068
:103530008FEF0895CF93DF9300D01F92CDB7DEB702
:103540009C0180918204843019F593E099833B8338
:103550002A839093E9008FEF9091E800815095FDC8
:1035600006C095ED9A95F1F700008111F5CF809195
:10357000E80085FF0DC040E050E063E070E0CE0160
:1035800001960E94E41C8091E8008E778093E80009
:103590000F900F900F90DF91CF910895CF93DF930D
:1035A00000D01F92CDB7DEB720918204243021F5E0
:1035B00022E029839B838A8383E08093E9008FEF55
:1035C0009091E800815095FD06C095ED9A95F1F730
:1035D00000008111F5CF8091E80085FF0DC040E02B
:1035E00050E063E070E0CE0101960E94E41C8091FF
:1035F000E8008E778093E8000F900F900F90DF9196
:10360000CF910895209182042430F1F422E0209398
:10361000E9002FEF3091E800215035FD06C035ED6F
:103620003A95F1F700002111F5CF2091E80025FF30
:103630000BC040E050E065E070E00E94E41C809127
:10364000E8008E778093E8000895CF93DF93209170
:103650008204243039F521E02093E9002FEF3091E6
:10366000E800215035FD06C035ED3A95F1F7000030
:103670002111F5CF2091E80025FF14C0EC0140E0B6
:1036800050E068E070E00E94E41C8091E8008E77D2
:103690008093E80088E0FE01A7EFB2E001900D9270
:1036A0008A95E1F7DF91CF91089585E892E00E9435
:1036B000C80280918104811109C00E94791E0E9474
:1036C000D61E8091E20084608093E200089581E834
:1036D00092E00E94C80210928104089508952091FA
:1036E000F4022F5F822F62E30E940632992319F0C1
:1036F0002093F40208951092F4028091F602882338
:1037000071F180918204843041F58091E9008F70DD
:103710002091EC00922F917020FD90E8892B94E08D
:103720009093E9009091EB0090FF14C09091EE000F
:1037300097FF10C09091E80095FF03C01092F10030
:10374000F9CF9091E80090FF05C09091E8009E7736
:103750009093E8008F708093E9001092F60208952C
:1037600042E061EC81E00E94F31D42E061EC82E006
:103770000E94F31D42E061EC83E00E94F31D42E2EF
:1037800061EC84E00C94F31D80918404833009F48F
:1037900053C030F4813071F0823009F48CC0089548
:1037A0008A3009F478C08B3009F45EC0893009F0A2
:1037B0009AC020C080918304813A09F094C080911E
:1037C000E800877F8093E8008091870490918804C7
:1037D000892B21F468E087EF92E003C060E080E08D
:1037E00090E070E00E942F1D8091E8008B7780931D
:1037F000E800089580918304813209F074C08091BB
:10380000870490918804892B09F06DC08091E800AD
:10381000877F8093E8008091E80082FD05C0809159
:1038200082048111F8CF5FC08091F1008093FF0284
:103830008091E8008B7753C080918304813A09F02E
:1038400052C08091870490918804892B09F04BC065
:103850008091E800877F8093E8008091E80080FFF6
:10386000FCCF80910A0136C0809183048132D9F562
:103870008091870490918804892BA9F58091E800B4
:10388000877F8093E8000E94281E809185048093A2
:103890000A010C94FE2680918304813221F58091E7
:1038A000E800877F8093E8000E94281E80918604AC
:1038B00080930003089580918304813AA1F480915C
:1038C000E800877F8093E8008091E80080FFFCCFCC
:1038D000809100038093F1008091E8008E778093BF
:1038E000E8000C94281E08958091FF028093F50251
:1038F0001092FF0280E00E94AF070E94DB220C942E
:10390000FE260C94741C0E94912D8091F5028093E8
:10391000FF0208950C94831C292F3327233031058F
:10392000C9F064F42130310581F02230310509F00D
:1039300043C084E790E02BED32E042C021323105F4
:10394000F1F02232310541F137C082E190E02FE4FD
:1039500033E036C099278130910541F082309105DE
:1039600041F0892B49F5E7EDF2E005C0E7ECF2E024
:1039700002C0E9E8F2E0849190E09F0121C0643048
:10398000D8F4E62FF0E0EE0FFF1FE057FE4F208146
:10399000318189E090E014C0643070F470E0FB0184
:1039A000EE0FFF1FE857FE4F20813181FB01EC57DE
:1039B000FE4F808190E004C080E090E020E030E0A5
:1039C000FA01318320830895CF92DF92EF92FF9224
:1039D0000F931F93CF93DF93EC018B016A010E9439
:1039E000471E811133C0C114D10439F0F601808122
:1039F0009181081B190BC80FD91FE12CF12C01155F
:103A0000110519F18091E80085FD16C08091E8004C
:103A10008E778093E800C114D10449F0F6018081CB
:103A20009181E80EF91EF182E08285E00FC00E94CC
:103A3000471E882321F30AC089918093F100015029
:103A40001109FFEFEF1AFF0ADACF80E0DF91CF9183
:103A50001F910F91FF90EF90DF90CF9008952091EC
:103A6000890430918A042617370748F061157105DB
:103A700039F42091E8002E772093E80001C0B901C5
:103A800040E061157105A9F120918204222309F417
:103A900043C0253009F442C02091E80023FD40C016
:103AA0002091E80022FD32C02091E80020FFE9CFFC
:103AB0004091F3002091F20030E0342BFC01CF0163
:103AC0006115710559F02830310540F481918093DA
:103AD000F100615071092F5F3F4FF1CF41E0283075
:103AE000310509F040E02091E8002E772093E800AE
:103AF000C8CF4111C9CF0AC080918204882361F0E8
:103B0000853061F08091E80083FD0AC08091E80073
:103B100082FFF2CF80E0089582E0089583E0089567
:103B200081E008952091890430918A04261737078F
:103B300048F06115710539F42091E8002E77209343
:103B4000E80001C0B901FC0120E06115710591F1A7
:103B500080918204882309F440C0853009F43FC075
:103B60008091E80083FD3DC08091E80082FD2FC078
:103B70008091E80080FFE9CF2091F3008091F2006E
:103B800090E0922B6115710559F08830910540F451
:103B900024912093F1003196615071090196F2CF82
:103BA00021E0089709F020E08091E8008E7780936B
:103BB000E800CBCF2111CCCF0AC0809182048823AA
:103BC00061F0853061F08091E80083FD0AC080914A
:103BD000E80082FFF2CF80E0089582E0089583E05C
:103BE000089581E00895982F973058F59093E90053
:103BF000981739F07091EC002091ED005091F00091
:103C000003C0242F762F50E021FF19C03091EB0024
:103C10003E7F3093EB003091ED003D7F3093ED001F
:103C20003091EB0031603093EB007093EC00209307
:103C3000ED005093F0002091EE0027FF07C09F5F3A
:103C4000D3CF8F708093E90081E0089580E00895DC
:103C50008091830487FF11C08091E80082FD05C038
:103C6000809182048111F8CF11C08091E8008B7798
:103C70000BC080918204882349F08091E80080FF86
:103C8000F8CF8091E8008E778093E8000895209126
:103C9000E4003091E50095E64091EC00842F8170BE
:103CA00040FF22C08091E80080FD1CC0809182040A
:103CB000882391F0853091F08091EB0085FD10C054
:103CC0004091E4005091E5004217530729F39A010F
:103CD000915011F784E0089582E0089583E00895FB
:103CE00081E0089580E008954091E80042FFDECF32
:103CF00008950E94E71E0E94EF1EE0EEF0E0808132
:103D000081608083E8EDF0E080818F77808319BC4B
:103D1000A7EDB0E08C918E7F8C9380818F7E808325
:103D20001092810408950F931F93CF93DF930E9405
:103D3000E71E0E94EF1EC8EDD0E088818F77888350
:103D400088818068888388818F7D888319BC1092E0
:103D5000820410927E041092800410927F0400EE80
:103D600010E0F80180818B7F808388818160888367
:103D700042E060E080E00E94F31DE1EEF0E080812F
:103D80008E7F8083E2EEF0E080818160808380819D
:103D900088608083F80180818E7F80838881806144
:103DA0008883DF91CF911F910F910895E8EDF0E0A6
:103DB00080818F7E8083E7EDF0E080818160808369
:103DC00084E082BF81E0809381040C94931EE8ED2F
:103DD000F0E080818E7F80831092E200089510923F
:103DE000DA001092E10008951F920F920FB60F9221
:103DF00011242F933F934F935F936F937F938F93F0
:103E00009F93AF93BF93EF93FF938091E10082FF65
:103E10000BC08091E20082FF07C08091E1008B7FA0
:103E20008093E1000E946F1B8091DA0080FF1FC029
:103E30008091D80080FF1BC08091DA008E7F809334
:103E4000DA008091D90080FF0DC080E189BD82E158
:103E500089BD09B400FEFDCF81E0809382040E94F9
:103E6000551B05C019BC109282040E94671B8091EB
:103E7000E10080FF19C08091E20080FF15C08091B1
:103E8000E2008E7F8093E2008091E2008061809367
:103E9000E2008091D80080628093D80019BC85E050
:103EA000809382040E94811C8091E10084FF30C0D5
:103EB0008091E20084FF2CC080E189BD82E189BD50
:103EC00009B400FEFDCF8091D8008F7D8093D8008B
:103ED0008091E1008F7E8093E1008091E2008F7EEF
:103EE0008093E2008091E20081608093E200809103
:103EF0007E04882311F084E007C08091E30087FDF1
:103F000002C081E001C083E0809382040E948A1C89
:103F10008091E10083FF29C08091E20083FF25C0EA
:103F20008091E100877F8093E10082E080938204AA
:103F300010927E048091E1008E7F8093E100809159
:103F4000E2008E7F8093E2008091E20080618093A6
:103F5000E20042E060E080E00E94F31D8091F0000A
:103F600088608093F0000E946E1BFF91EF91BF91DB
:103F7000AF919F918F917F916F915F914F913F9101
:103F80002F910F900FBE0F901F9018951F920F92B8
:103F90000FB60F9211242F933F934F935F936F931C
:103FA0007F938F939F93AF93BF93CF93DF93EF93C1
:103FB000FF93C091E900CF708091EC00D82FD170B1
:103FC00080FDD0E81092E9008091F000877F809317
:103FD000F00078940E940A201092E9008091F0008D
:103FE00088608093F000CD2BCF70C093E900FF91E3
:103FF000EF91DF91CF91BF91AF919F918F917F9181
:104000006F915F914F913F912F910F900FBE0F9045
:104010001F9018951F93CF93DF93CDB7DEB7AA9764
:104020000FB6F894DEBF0FBECDBFE3E8F4E088E042
:104030008E0F9091F10091938E13FBCF0E94C41BC1
:104040008091E80083FF1FC18091830490918404D4
:10405000492F50E04A30510508F015C1FA01EA5ADB
:10406000FF4F0C942632803881F0823809F00BC162
:10407000809187048F708093E9008091EB0085FB2D
:10408000882780F91092E90006C080917F04909102
:104090008004911182609091E800977F9093E800EE
:1040A0008093F1001092F100C8C0282F2D7F09F0F5
:1040B000EAC0882319F0823061F0E5C08091850460
:1040C000813009F0E0C0933009F080E080938004F3
:1040D0002BC080918504811127C0809187048F7047
:1040E00009F4D1C08093E9002091EB0020FF1CC0AF
:1040F000933021F48091EB00806214C09091EB002A
:1041000090619093EB0021E030E0A90102C0440FE0
:10411000551F8A95E2F74093EA001092EA008091D9
:10412000EB0088608093EB001092E9008091E8003A
:10413000877F86C08111A7C0109185041F77809169
:10414000E3008078812B8093E3008091E800877FF3
:104150008093E8000E94281E8091E80080FFFCCF39
:104160008091E30080688093E300111102C082E037
:1041700001C083E08093820486C08058823008F0BA
:1041800082C080918504909186048C3D53E0950710
:1041900079F583E08A838AE289834FB7F894DE0158
:1041A000139620E03EE051E2E32FF0E050935700F9
:1041B000E49120FF03C0E295EF703F5FEF708E2F18
:1041C00090E0EA3010F0C79601C0C0968D939D93A1
:1041D0002F5F243149F74FBF8091E800877F80939C
:1041E000E8006AE270E0CE0101960E942F1D14C023
:1041F000AE014F5F5F4F609187040E948C1CBC0131
:10420000892B09F440C09091E800977F9093E800D3
:1042100089819A810E94921D8091E8008B7780931A
:10422000E80031C0803879F58091E800877F80937D
:10423000E80080917E048093F1008091E8008E7701
:104240008093E8000E94281E1EC081111CC090911E
:1042500085049230C0F48091E800877F8093E80065
:1042600090937E040E94281E80917E04811106C0D6
:104270008091E30087FD02C081E001C084E080936B
:1042800082040E94B01B8091E80083FF0AC08091E5
:10429000E800877F8093E8008091EB008062809344
:1042A000EB00AA960FB6F894DEBF0FBECDBFDF912C
:1042B000CF911F910895909306038093050308956D
:1042C000E0910503F0910603309721F00190F08111
:1042D000E02D099480E00895EF92FF920F931F93D1
:1042E000CF93DF93E0910503F09106033097B1F18E
:1042F0008C010280F381E02D09958091730482FF87
:104300002DC080FF04C08CE694E00E94C802E80142
:1043100018E086E6E82E84E0F82E8091730480FF92
:104320000BC088811F928F93FF92EF920E946103CE
:104330000F900F900F900F90115021961111EDCF0B
:104340008091730480FF0AC084E694E0DF91CF91EE
:104350001F910F91FF90EF900C94C802DF91CF91C5
:104360001F910F91FF90EF900895E0910503F09158
:104370000603309721F00480F581E02D099408951B
:10438000CF93DF93EC018091030390910403C8174E
:10439000D90709F1D0930403C0930303E091050307
:1043A000F09106033097B9F00680F781E02DCE0139
:1043B00009958091730482FF0EC080FF0CC0DF93CB
:1043C000CF9386E594E09F938F930E9461030F90B3
:1043D0000F900F900F90DF91CF910895CF93DF93BF
:1043E000EC018091010390910203C817D90709F1EC
:1043F000D0930203C0930103E0910503F0910603FB
:104400003097B9F00084F185E02DCE0109958091B7
:10441000730482FF0EC080FF0CC0DF93CF9386E44D
:1044200094E09F938F930E9461030F900F900F90E1
:104430000F90DF91CF9108950E94600B0C94DB08E0
:104440008F929F92AF92BF92CF92DF92EF92FF92A4
:104450000F931F93CF93DF9300D000D01F92CDB75F
:10446000DEB70E94130608E013E0F12C8F2D0E94A6
:1044700045074C01F801A080B180A826B926A114F7
:10448000B10439F4F3940E5F1F4FF0E1FF12EECF49
:1044900039C08091730481FD0E947507E12CCC2402
:1044A000C394D12CC6018A219B21892B21F1E98259
:1044B000FA8221E0C60188219921892B09F420E0A4
:1044C0002B830E94690B8160782F9D838C834981A7
:1044D0005A816B818D810E94DC2249815A816B81D6
:1044E0007C818D810E947E2DF801808191818C25B7
:1044F0009D2591838083E394CC0CDD1CF0E1EF12C9
:10450000D1CFC0CF8FEF89838A831B820E94690B32
:104510008160782F9D838C8349815A816B818D8145
:104520000E94DC220E947D2D0E94F62F109107032D
:104530000E946021181759F10E946021809307039F
:104540009091730492FF0EC090FF0CC01F928F9346
:1045500087E794E09F938F930E9461030F900F90E1
:104560000F900F90809107030F900F900F900F9076
:104570000F90DF91CF911F910F91FF90EF90DF90FF
:10458000CF90BF90AF909F908F900C948F2D0F90F5
:104590000F900F900F900F90DF91CF911F910F917F
:1045A000FF90EF90DF90CF90BF90AF909F908F9053
:1045B00008950C94AF070895CF93DF93CDB7DEB77E
:1045C0002B970FB6F894DEBF0FBECDBF942F4F834D
:1045D000252F588769877A878B874A855B85452B86
:1045E00021F02F3F09F59F3FF9F4DE01119686E097
:1045F000FD0111928A95E9F785E0FE013796019059
:104600000D928A95E1F749815A816B817C818D8178
:104610009E810E94DB292B960FB6F894DEBF0FBE59
:10462000CDBFDF91CF9108954F81588569857A85F7
:104630008B850E947E2DD9CF882309F45CC09CEF26
:10464000980F913A20F090E5980F9E3218F40E944E
:10465000A92C0DC090E2980F983058F4877091E023
:1046600001C0990F8A95EAF7892F0E94E82C0C94D3
:10467000222D9BE5980F933070F4853A29F0863A05
:1046800031F083E890E005C081E890E002C082E864
:1046900090E00C94C02198E5980F953160F5883A28
:1046A00089F0893A91F08A3A99F08B3AA1F08C3AE4
:1046B000A9F08D3AB1F08E3AB9F08F3AC1F080E0AE
:1046C00090E017C082EE90E014C089EE90E011C037
:1046D0008AEE90E00EC085EB90E00BC086EB90E098
:1046E00008C083EB90E005C084EB90E002C087EB4C
:1046F00090E00C94EE210895882349F19CEF980FE7
:10470000913A20F090E5980F9E3218F40E94C62C42
:104710000DC090E2980F983058F4877091E001C076
:10472000990F8A95EAF7892F0E94EE2C0C94222D7E
:104730009BE5980F933020F480E090E00C94C0212A
:10474000885A853120F480E090E00C94EE210895A1
:10475000882321F00E94E82C0C94222D08958823B0
:1047600021F00E94EE2C0C94222D0895BF92CF923E
:10477000DF92EF92FF920F931F93CF93DF9300D0BE
:1047800000D000D0CDB7DEB725E0FC01DE011196E8
:1047900001900D922A95E1F7FC014081518102813F
:1047A00063817481258122952F706115710509F44B
:1047B00003C35F3F19F44F3F09F4FEC26C01862F1B
:1047C0007D836C83602F782F8D812E830E942D2C0A
:1047D000182FB92E0E942C2C0E94262BEB2DE2952F
:1047E000EF70F0E0E05AFF4F2E810C9426328B2DB3
:1047F000807F9B2D9F70F92E882319F0F29490EF03
:10480000F922002349F0FF2009F483C28F2D0E9472
:10481000FB2C0E94222D7DC2812F0E947C23FF2031
:1048200009F4CAC28F2D0E94012D26960FB6F89466
:10483000DEBF0FBECDBFDF91CF911F910F91FF90D3
:10484000EF90DF90CF90BF900C94222D8B2D807F26
:104850009B2D9F70F92E803219F0F29480EFF82290
:10486000112319F0113009F12AC00023B1F08F2D66
:10487000222351F1213041F526960FB6F894DEBF80
:104880000FBECDBFDF91CF911F910F91FF90EF90A1
:10489000DF90CF90BF900C940B2D222319F0213084
:1048A00009F48AC20E940E2D2DC00023F1F026309B
:1048B00008F082C20E94E52C8F2129F023C000233A
:1048C000F9F0211116C08F2D26960FB6F894DEBF91
:1048D0000FBECDBFDF91CF911F910F91FF90EF9051
:1048E000DF90CF90BF900C94A823253008F064C2CD
:1048F00009C0F601858180FF0CC28F708583E3CFEC
:1049000021111CC28F2D83C12B2D26952695237036
:1049100030E02115310521F021303105D1F04CC2B4
:10492000002321F0812F9B2D937002C080E090E046
:1049300026960FB6F894DEBF0FBECDBFDF91CF91A4
:104940001F910F91FF90EF90DF90CF90BF900C944C
:10495000C021002321F0812F9B2D937002C080E0A5
:1049600090E026960FB6F894DEBF0FBECDBFDF9164
:10497000CF911F910F91FF90EF90DF90CF90BF905C
:104980000C94EE21812F002319F00E947C2E02C08E
:104990000E94E42E26960FB6F894DEBF0FBECDBF60
:1049A000DF91CF911F910F91FF90EF90DF90CF900B
:1049B000BF900C94692F8B2D837009F07BC001117F
:1049C000FBC1812F829586958770880F880F912F64
:1049D0009F70C92ED12CE12CF12C082E04C0CC0CD8
:1049E000DD1CEE1CFF1C0A94D2F714FF12C04FE02E
:1049F00050E060E070E004C0440F551F661F771F51
:104A00008A95D2F7CB01BA01609570958095909503
:104A100003C060E070E0CB012B2D26952695237016
:104A2000422F50E042305105D9F04330510569F131
:104A30006C297D298E299F294130510551F12696F7
:104A40000FB6F894DEBF0FBECDBFDF91CF911F919F
:104A50000F91FF90EF90DF90CF90BF900C94412B7F
:104A60006C297D298E299F2926960FB6F894DEBFE2
:104A70000FBECDBFDF91CF911F910F91FF90EF90AF
:104A8000DF90CF90BF900C945B2B0E94412BC7010D
:104A9000B60126960FB6F894DEBF0FBECDBFDF91EC
:104AA000CF911F910F91FF90EF90DF90CF90BF902B
:104AB0000C94272B002319F08B2D817001C0869553
:104AC000882309F479C1812F829586958770880F94
:104AD000880F912F9F70C92ED12CE12CF12C082E1C
:104AE00004C0CC0CDD1CEE1CFF1C0A94D2F714FF92
:104AF00012C04FE050E060E070E004C0440F551F6A
:104B0000661F771F8A95D2F7CB01BA016095709521
:104B10008095909503C060E070E0CB012B2D269529
:104B200026952370422F50E042305105D9F0433092
:104B3000510569F16C297D298E299F294130510544
:104B400051F126960FB6F894DEBF0FBECDBFDF91B0
:104B5000CF911F910F91FF90EF90DF90CF90BF907A
:104B60000C94082C6C297D298E299F2926960FB636
:104B7000F894DEBF0FBECDBFDF91CF911F910F9193
:104B8000FF90EF90DF90CF90BF900C941A2C0E9472
:104B9000082CC701B60126960FB6F894DEBF0FBEEB
:104BA000CDBFDF91CF911F910F91FF90EF90DF90DC
:104BB000CF90BF900C94F62B103FD1F128F480E4F5
:104BC000810F803250F0A0C0123F09F462C008F497
:104BD0004BC0133F09F472C097C0F12FF071FF2E44
:104BE0008B2D8F71002351F00E948F2B812FFF207E
:104BF00019F08295807F68CE8F7066CE0E94B02BB0
:104C0000812FFF2019F08295807F01C08F7026963A
:104C10000FB6F894DEBF0FBECDBFDF91CF911F91CD
:104C20000F91FF90EF90DF90CF90BF900C94AF2347
:104C30000023B1F0253008F0BFC08B2D8F71269670
:104C40000FB6F894DEBF0FBECDBFDF91CF911F919D
:104C50000F91FF90EF90DF90CF90BF900C94D52BE9
:104C6000263008F0A9C0E9CF0023A9F08B2D8F7161
:104C700026960FB6F894DEBF0FBECDBFDF91CF9161
:104C80001F910F91FF90EF90DF90CF90BF900C9409
:104C90008F2B002359F38B2D8F7126960FB6F89426
:104CA000DEBF0FBECDBFDF91CF911F910F91FF905F
:104CB000EF90DF90CF90BF900C94B02B002399F031
:104CC0008B2D8F7126960FB6F894DEBF0FBECDBF29
:104CD000DF91CF911F910F91FF90EF90DF90CF90D8
:104CE000BF900C947A2B26960FB6F894DEBF0FBEB9
:104CF000CDBFDF91CF911F910F91FF90EF90DF908B
:104D0000CF90BF900C94752B0023A9F0222309F4B7
:104D1000ADCF812F26960FB6F894DEBF0FBECDBF64
:104D2000DF91CF911F910F91FF90EF90DF90CF9087
:104D3000BF900C941C23222309F4ADCF812F26961B
:104D40000FB6F894DEBF0FBECDBFDF91CF911F919C
:104D50000F91FF90EF90DF90CF90BF900C947C2349
:104D60004B2D4F70612FC6010E94F62D26960FB66F
:104D7000F894DEBF0FBECDBFDF91CF911F910F9191
:104D8000FF90EF90DF90CF90BF900C947F2A4B2D37
:104D90004F70612FC60126960FB6F894DEBF0FBE86
:104DA000CDBFDF91CF911F910F91FF90EF90DF90DA
:104DB000CF90BF900C94F92D26960FB6F894DEBFD5
:104DC0000FBECDBFDF91CF911F910F91FF90EF905C
:104DD000DF90CF90BF9008950E94082D0E94D72C9D
:104DE0000E94222D0E949B300E94692F80E090E05B
:104DF0000E94C02180E090E00C94EE210E94F82CEB
:104E00000C94EC26CF93DF9300D000D01F92CDB747
:104E1000DEB7942F4983252F5A836B837C838D8340
:104E20004C815D81452B39F12F3F11F49F3F19F1E2
:104E300049815A816B817C818D810E942D2C292F83
:104E400022952F7030E02C30310504F52A303105E1
:104E50005CF4225031092230310568F4853A80F43F
:104E6000843090F4823080F0883E38F4803E60F4E4
:104E70008450813A48F080E014C0803FE1F704C0DC
:104E800090E2980F983080F781E00BC02C3031050C
:104E900021F493FB882780F904C02F303105C9F332
:104EA000EACF0F900F900F900F900F90DF91CF915E
:104EB0000895CF93DF9300D000D01F92CDB7DEB717
:104EC0000F900F900F900F900F90DF91CF9108955A
:104ED000CF93DF9300D000D000D0CDB7DEB72696B9
:104EE0000FB6F894DEBF0FBECDBFDF91CF9108950E
:104EF0001F93CF93DF93C091280316E0809129037D
:104F0000C81799F0D0E01C9FF0011D9FF00D1124EF
:104F1000E65DFC4F4081518162817381848195817E
:104F20000E9468272196C770E9CFDF91CF911F912A
:104F3000089540915A0350915B0360915C03709116
:104F40005D0380915E0390915F030C9468278091CC
:104F50005F0382958F7009F054C080915C038823B1
:104F600009F44FC080912803A091290360915A034E
:104F700070915B0340915D0350915E03B6E08A1728
:104F800009F43FC090E041155105C1F17F3F11F494
:104F90006F3FA1F1B89FF001B99FF00D1124E65DBC
:104FA000FC4F218172132AC02081621327C0228105
:104FB000211124C0238134812417350710F4215096
:104FC0003109241B350B283C3105C0F420915F03C7
:104FD0002F70206120935F0326E0289FF001299F16
:104FE000F00D1124E15DFC4F80818F708061808322
:104FF0008AE593E00E94B6230C9478270196877087
:10500000BECF0895BF92CF92DF92EF92FF920F939F
:105010001F93CF93DF93CDB7DEB761970FB6F894A8
:10502000DEBF0FBECDBF7C0185E0F701DE011D961E
:1050300001900D928A95E1F7D7014C9111965C9100
:1050400011971296DC90129713960D911C9114975C
:1050500030915A0360915B0380915D0390915E03F0
:10506000009709F477C16F3F19F43F3F09F472C10B
:10507000B0905C03BB2009F4C5C020915F03081702
:10508000190728F0F801E81BF90BCF0104C080953F
:105090009095800F911FCC24C394883C910580F09B
:1050A000C12C207F09F0CCC0702F198B088B6D2D7F
:1050B00089890E9459278AE593E00E94B623B6C0E9
:1050C000822F807F09F047C0651314C0341312C0CB
:1050D000D11010C02F70206120935F030E94992788
:1050E0008AE593E00E94B62380915F03D70115966D
:1050F0008C932FC00115110519F15F3F11F44F3F3B
:10510000F9F0CD2CD1101CC08091280320912903E7
:1051100036E0821709F45CC090E0389FF001399FB7
:10512000F00D1124E65DFC4F6181561306C06081CD
:10513000461303C06281611103C001968770E9CFF5
:10514000CD2CDD2009F426C180915F03816080931E
:105150005F03C12C1FC1651308C0341306C0D110F2
:1051600004C080915F03D701C9C04D875E87DF8689
:10517000702F198B088B6D2D89890E940227882337
:10518000E9F1DD20D9F120915F03822F82958F70A4
:1051900090E0029774F080915A0390915B03988796
:1051A0008F8319861B870A872C87CE0107960E945A
:1051B000B62386E0F701AAE5B3E001900D928A9547
:1051C000E1F70E94A7270E949927CC24C394E2C04C
:1051D000702F198B088B60E089890E942D2C292F54
:1051E00022952F7030E0223031050CF0C7C09F703F
:1051F00009F0C1C0805E883008F4CCC0C7010E94AD
:10520000B623E3CF0817190708F456C0F801E81BC6
:10521000F90BCF01883C910508F453C0C12C702FC5
:10522000198B088B6D2D89890E945927EAE5F3E0D7
:1052300086E0DF011D928A95E9F70E949927AAC0AE
:10524000651314C0341312C0D11010C080915F03D5
:10525000F7018583C7010E94B62386E0EAE5F3E003
:10526000DF011D928A95E9F7CB2C94C04D875E87AC
:10527000DF86702F198B088B6D2D89890E9402277C
:10528000882309F4BBCFDD2009F4B8CF20915F0358
:10529000822F82958F7090E002970CF48ACF8091D4
:1052A0005A0390915B039A8389831B821D830C832D
:1052B0002E83CE0101967BCF80959095800F911F14
:1052C000A9CFCD2CDD2009F499CF65132EC034135E
:1052D0002CC020915F0320FD1FC0822F82958F700C
:1052E000D9F0D70115962C9315978F3049F08F5F21
:1052F000982F9295907F822F8F70892B15968C9383
:10530000C7010E94B62386E0F701AAE5B3E0019049
:105310000D928A95E1F791CF86E0F701AAE5B3E017
:1053200001900D928A95E1F735C04D875E87DF8643
:10533000702F198B088B6D2D89890E94022781118E
:1053400038CF80915F03816080935F03C7010E9423
:10535000B62320C0DD2009F451CF4D875E87DF865C
:10536000702F198B088B6D2D89890E940227882345
:1053700009F444CF1ECF81113DCF0CC0243031053C
:105380000CF03CCF9F7009F435CFF7019581907FE9
:1053900009F030CF8C2D61960FB6F894DEBF0FBEAA
:1053A000CDBFDF91CF911F910F91FF90EF90DF90D4
:1053B000CF90BF9008951F93CF93DF93CDB7DEB703
:1053C0002C970FB6F894DEBF0FBECDBF4F83588722
:1053D00069877A878B879C87CE0107960E9402286F
:1053E000882369F08F8198852A853B85232BF1F1ED
:1053F0009F3F09F063C08F3F09F060C037C086E06F
:10540000FE013796DE01119601900D928A95E1F723
:105410006F817885EA85FB85309741F17F3F11F4F4
:105420006F3F21F12091290330E0C9010196877077
:1054300099274091280350E08417950709F447C045
:1054400069837A83FD83EC8396E0929FD001939FDA
:10545000B00D1124A65DBC4FFE01319601900D9256
:105460009A95E1F7809329030E94782716E08091AE
:105470002803909129038917C1F1189FC0011124B5
:10548000865D9C4F0E940228882379F1E0912803D1
:105490001E9FF0011124E65DFC4F40815181628125
:1054A0007381848195810E9468278091280390E010
:1054B00001968770992780932803D9CF4F8158850B
:1054C00069857A858B859C850E946827CFCF0E944D
:1054D000FE261092290310922803EAE5F3E086E005
:1054E000DF011D928A95E9F7C1CF2C960FB6F8948B
:1054F000DEBF0FBECDBFDF91CF911F910895DF9228
:10550000EF92FF920F931F93CF93DF93FC01892BB0
:1055100009F48AC0E12CF12CDD24D394EF0121960B
:105520008491853709F461C058F4843708F04EC07F
:10553000843008F06AC08130D1F0823071F174C0DB
:10554000883709F45DC050F4863709F455C08737B1
:1055500009F06AC08E2D0E94F52C54C09CE7980F6C
:10556000903708F061C08F770E947C2350C08F0174
:105570000E5F1F4FFE01849190E2980F983050F417
:105580008770FD2D01C0FF0F8A95EAF78F2F0E94CB
:10559000FB2C14C00E941C2313C08F010E5F1F4FF1
:1055A000FE01C49180E28C0F883060F4C7708D2DAD
:1055B00001C0880FCA95EAF70E94012D0E94222D92
:1055C000E80125C08C2F0E947C23FACF9F012E5F1B
:1055D0003F4FFE01C491CC2369F08FE99FE0019712
:1055E000F1F700C00000C150F6CF9F012E5F3F4F82
:1055F000FE01F490E9010BC00E94E52CE82E07C0E3
:105600000E94F82C0E94222D02C00E941C238F2D84
:10561000882341F0EFE9FFE03197F1F700C0000087
:105620008150F6CFFE017ACFDF91CF911F910F917C
:10563000FF90EF90DF900895609360047093610491
:1056400080936204909363040C948E2D08950F93BD
:105650001F930091640410916504209166043091B9
:105660006704602B712B822B932B609364047093DF
:10567000650480936604909367041F910F910C94C6
:105680008D2D0F931F930091640410916504209158
:10569000660430916704602371238223932360930F
:1056A00064047093650480936604909367041F916B
:1056B0000F910C948D2D0F931F9300916404109102
:1056C0006504209166043091670460277127822762
:1056D00093276093640470936504809366049093A9
:1056E00067041F910F910C948D2D60E070E0CB0149
:1056F0000C941C2B0F931F9341E050E060E070E08E
:105700008A019B0104C0000F111F221F331F8A95BD
:10571000D2F7C901B8011F910F910C941C2B0F9364
:105720001F9341E050E060E070E004C0440F551F5B
:10573000661F771F8A95D2F780916004909161046B
:10574000A0916204B09163048A019B01082B192B7C
:105750002A2B3B2BC901B8011F910F910C941C2BD4
:105760000F931F9341E050E060E070E004C0440FED
:10577000551F661F771F8A95D2F740955095609503
:1057800070958091600490916104A0916204B09141
:1057900063048A019B01082319232A233B23C9019F
:1057A000B8011F910F910C941C2B0F931F9341E094
:1057B00050E060E070E004C0440F551F661F771F83
:1057C0008A95D2F78091600490916104A09162045F
:1057D000B09163048A019B01082719272A273B27D8
:1057E000C901B8011F910F910C941C2B0F931F93AB
:1057F000009160041091610420916204309163046F
:10580000602B712B822B932B1F910F910C941C2BCF
:105810000F931F9300916004109161042091620422
:105820003091630460237123822393231F910F918E
:105830000C941C2B0F931F93009160041091610432
:105840002091620430916304602771278227932797
:105850001F910F910C941C2B08958F929F92AF92E1
:10586000BF92DF92EF92FF920F931F93CF93DF933C
:1058700000D000D01F92CDB7DEB76B837C838D83C1
:105880008A018C819D81892B21F01F3F29F44F3F94
:1058900019F480E090E04CC08B818823C9F180909E
:1058A000640490906504A0906604B09067048091B1
:1058B000600490916104A0916204B0916304882A0D
:1058C000992AAA2ABB2A8FE1E82EF12CD501C4011E
:1058D0000E2C04C0B695A795979587950A94D2F794
:1058E00080FF07C0DE2CB8018E2D0E94CC2D0197C1
:1058F00029F481E0E81AF10848F7D12C80E1189FDB
:10590000F0011124E00FF11DE05AFC4FD08209C0D4
:1059100080E1189FF0011124E00FF11DE05AFC4FC7
:10592000D08009831A8369817A818D2D0E94CC2DC4
:105930000F900F900F900F900F90DF91CF911F91CC
:105940000F91FF90EF90DF90BF90AF909F908F905E
:10595000089520910B0130910C01F90132969FEFCF
:1059600040E05191581789F09F3F19F4511101C03F
:10597000942F4F5F4630A9F79F3F39F0F901E90FA7
:10598000F11D97FDFA9582830895089520910B01EA
:1059900030910C01F9013296285F3F4F90819813A6
:1059A00001C010823196E217F307C1F7089581E034
:1059B00090E0E0910B01F0910C01E80FF91F1082CB
:1059C000019688309105A9F7089580917204089591
:1059D00090917204892B8093720408958095909120
:1059E0007204892380937204089580937204089549
:1059F00010927204089590917104892B8093710420
:105A0000089580959091710489238093710408957D
:105A100010927104089580936804089510926804A8
:105A2000089580910B0190910C01FC0131969C012D
:105A3000285F3F4F80E0919191118F5FE217F3074C
:105A4000D1F70895E0910B01F0910C01809172045F
:105A50008083E0910B01F0910C01908180917104A1
:105A6000892B808380916804882361F0E0910B0189
:105A7000F0910C019081892B80830E94112D81115E
:105A80001092680480910B0190910C010C946C2190
:105A9000909399018093980108958295982F9C7C0A
:105AA000392F36953695282F237344E0249FC00163
:105AB0001124932F982B292F2A7A2695892F8575C3
:105AC000880F822B08951F93CF93DF931F92CDB73A
:105AD000DEB799830E944D2D182F9981892F0E943E
:105AE0004D2D212F30E0322F2227A901482BCA014A
:105AF0000F90DF91CF911F9108950895CF93DF9379
:105B000000D000D01F92CDB7DEB70F900F900F904E
:105B10000F900F90DF91CF910895089508950C9400
:105B2000D9220E94DB220C94FE261F920F920FB600
:105B30000F9211248F939F93AF93BF93809174041E
:105B4000811113C08091E8029091E902A091EA02CC
:105B5000B091EB024196A11DB11D8093E802909394
:105B6000E902A093EA02B093EB02BF91AF919F913B
:105B70008F910F900FBE0F901F90189520E1929F6C
:105B8000F0011124E80FF11DE052FF4F9491892F8D
:105B90008F7092959F700895CF93C82FCB010E946C
:105BA000BE2D282F30E080E1989FA0011124422BC8
:105BB000532B4038510519F480E090E015C09770E0
:105BC000E92FF0E088E0C89FE00DF11D112484E08A
:105BD000EE0FFF1F8A95E1F7E20FF31FEE0FFF1F95
:105BE000E050F84985919491CF91089580E090E03C
:105BF000089508958091770480FF0BC06091100193
:105C000085E0689FB0011124759567957595679536
:105C10002BC081FF09C06091100185E0689FB00131
:105C200011247595679520C082FF07C0609110010F
:105C300085E0689FB001112417C0909178049923E2
:105C4000D1F060910F01961788F72091100185E03F
:105C5000289F90011124929FA001939F500D112421
:105C600070E0CA010E9412326038710540F461157B
:105C7000710539F002C065E070E0862F08958FE766
:105C8000089581E008958091770480FF08C06091B5
:105C90000E0170E0759567957595679521C081FF38
:105CA00006C060910E0170E07595679519C082FF7E
:105CB00004C060910E0170E010C0909178049923A7
:105CC000C1F060910D019617A0F780910E01899F98
:105CD000C001112470E00E9412326038710528F46E
:105CE0006115710521F0862F08958FE7089581E0F1
:105CF000089561E070E0F4CF803F21F40E94FA2D16
:105D0000819504C0813F29F40E94FA2D80937B0481
:105D10000895823F21F40E94FA2D819504C0833FAB
:105D200029F40E94FA2D80937A040895893F19F48A
:105D30000E94432E05C08A3F31F40E94432E819574
:105D400080937C0408958B3F21F40E94432E81951B
:105D500004C08C3F29F40E94432E80937D04089553
:105D6000843F21F480917904816017C0853F21F43C
:105D700080917904826011C0863F21F4809179047A
:105D800084600BC0873F21F480917904886005C04E
:105D9000883F31F48091790480618093790408957B
:105DA0008D3F21F48091770481600BC08E3F21F4F8
:105DB00080917704826005C08F3F29F48091770439
:105DC0008460809377040895803F39F480917B0448
:105DD00087FF6CC010927B0469C0813F29F48091D9
:105DE0007B041816BCF362C090917A04823F29F4B8
:105DF00097FF5CC010927A0459C0833F19F41916BA
:105E0000CCF354C0893F41F480917C0418160CF007
:105E10004DC010927C044AC08A3F29F480917C04D2
:105E200087FF44C0F6CF8B3F39F480917D0487FF14
:105E30003DC010927D043AC08C3F29F480917D04CE
:105E40001816BCF333C0843F21F4809179048E7F0F
:105E500017C0853F21F4809179048D7F11C0863F62
:105E600021F4809179048B7F0BC0873F21F48091CE
:105E70007904877F05C0883F31F4809179048F7E53
:105E80008093790413C08D3F21F4809177048E7F35
:105E90000BC08E3F21F4809177048D7F05C08F3F2A
:105EA00029F4809177048B7F8093770480917A0422
:105EB00081110EC080917B0481110AC080917C0405
:105EC000811106C080917D04811102C01092780476
:105ED00008958091730483FF7EC089EA94E00E9454
:105EE000C802809179041F928F9384EA94E09F9373
:105EF0008F930E94610382EA94E00E94C80280911D
:105F00007A04282F082E000C330B3F938F938FE9D0
:105F100094E09F938F930E9461038DE994E00E9427
:105F2000C80280917B04282F082E000C330B3F936E
:105F30008F938AE994E09F938F930E94610388E98D
:105F400094E00E94C80280917C04282F082E000C47
:105F5000330B3F938F9385E994E09F938F930E9437
:105F6000610383E994E00E94C80280917D04282F98
:105F7000082E000C330B3F938F9380E994E09F939E
:105F80008F930E9461038DE894E00E94C802809183
:105F900078041F928F938AE894E09F938F930E94D6
:105FA000610388E894E00E94C802809177041F9200
:105FB0008F9385E894E09F938F930E94610382E81A
:105FC00094E00E94C8028DB79EB74C960FB6F89425
:105FD0009EBF0FBE8DBF89E794E00E94B5210E944D
:105FE000690B909376048093750408951F93CF9363
:105FF000DF9380917504909176040E94810BAC012F
:1060000090917804992321F02091110130E006C08D
:10601000209112018AE0289F900111244217530712
:1060200008F485C080917A04C0917B04D0917C04EF
:1060300010917D04811107C0C11175C0D11173C0C9
:10604000111171C074C09F3F19F09F5F9093780445
:10605000181624F40E94FA2D80937A0480917A0411
:1060600087FF05C00E94FA2D819580937A041C1643
:1060700024F40E94FA2D80937B0480917B0487FF97
:1060800005C00E94FA2D819580937B0460917A046B
:10609000662331F1C0917B04CC2311F1062E000C54
:1060A000770B880B990B0E94E43023E333E343E33F
:1060B0005FE30E9499310E94AC3060937A046C2FA8
:1060C000CC0F770B880B990B0E94E43023E333E36A
:1060D00043E35FE30E9499310E94AC3060937B04FC
:1060E0001D1624F40E94432E80937C0480917C042E
:1060F00087FF05C00E94432E819580937C04111672
:1061000024F40E94432E80937D0480917D0487FFB8
:1061100005C00E94432E819580937D04DF91CF912D
:106120001F910C94692F9F3F09F08FCF97CFDF917C
:10613000CF911F910895E9E7F4E085E0DF011D921A
:106140008A95E9F7109278041092770408950E94D6
:106150001F3108F481E008950E94B3306894B111B2
:106160000C948E3108950E94733188F09F5798F0F7
:10617000B92F9927B751B0F0E1F0660F771F881F4C
:10618000991F1AF0BA95C9F714C0B13091F00E9466
:106190008D31B1E008950C948D31672F782F8827C9
:1061A000B85F39F0B93FCCF3869577956795B3958D
:1061B000D9F73EF490958095709561957F4F8F4FFC
:1061C0009F4F0895E89409C097FB3EF49095809501
:1061D000709561957F4F8F4F9F4F9923A9F0F92FAD
:1061E00096E9BB279395F695879577956795B7952B
:1061F000F111F8CFFAF4BB0F11F460FF1BC06F5F11
:106200007F4F8F4F9F4F16C0882311F096E911C022
:10621000772321F09EE8872F762F05C0662371F043
:1062200096E8862F70E060E02AF09A95660F771F57
:10623000881FDAF7880F9695879597F90895990F33
:106240000008550FAA0BE0E8FEEF16161706E80740
:10625000F907C0F012161306E407F50798F0621B61
:10626000730B840B950B39F40A2661F0232B242B36
:10627000252B21F408950A2609F4A140A6958FEF55
:10628000811D811D089597F99F6780E870E060E0A7
:1062900008959FEF80EC089500240A9416161706BF
:1062A00018060906089500240A9412161306140607
:1062B00005060895092E0394000C11F4882352F06A
:1062C000BB0F40F4BF2B11F460FF04C06F5F7F4F22
:1062D0008F4F9F4F089557FD9058440F551F59F009
:1062E0005F3F71F04795880F97FB991F61F09F3FC3
:1062F00079F087950895121613061406551FF2CFEC
:106300004695F1DF08C0161617061806991FF1CF3B
:1063100086957105610508940895E894BB27662762
:106320007727CB0197F908950E941F3108F48FEF6A
:1063300008950E94AC310C945A310E944C3138F0CF
:106340000E94533120F0952311F00C9443310C94AA
:10635000493111240C948E310E946B3170F3959F5A
:10636000C1F3950F50E0551F629FF001729FBB274C
:10637000F00DB11D639FAA27F00DB11DAA1F649FE8
:106380006627B00DA11D661F829F2227B00DA11D9B
:10639000621F739FB00DA11D621F839FA00D611D21
:1063A000221F749F3327A00D611D231F849F600D42
:1063B000211D822F762F6A2F11249F5750409AF06B
:1063C000F1F088234AF0EE0FFF1FBB1F661F771FF7
:1063D000881F91505040A9F79E3F510580F00C94C2
:1063E00043310C948E315F3FE4F3983ED4F38695AD
:1063F00077956795B795F795E7959F5FC1F7FE2B62
:10640000880F911D9695879597F90895991B79E0C6
:1064100004C0991F961708F0961B881F7A95C9F734
:106420008095089597FB072E16F4009407D077FD0A
:1064300009D00E942C3207FC05D03EF4909581953E
:106440009F4F0895709561957F4F0895EE0FFF1F40
:106450000590F491E02D0994AA1BBB1B51E107C0E4
:10646000AA1FBB1FA617B70710F0A61BB70B881FE4
:10647000991F5A95A9F780959095BC01CD01089573
:04648000F894FFCFBE
:10648400341A251B021BCE1A9A1A0169042808140F
:106494000A321E66756C6C006C6F77000000000099
:1064A400DB09000000002C04000000009B046A03C8
:1064B400B9032D04D4036C036D03D703DC03E10398
:1064C400AD03B603E903FEFF000022040000000050
:1064D400790A00000000F90A0C1AEF0AF50AF20A18
:1064E400F80AEE0A000000007A0CD00B920C0000AF
:1064F4000000B9166A031816A919101608186D03B6
:1065040013166F03404D36220604B9038303610357
:08651400ED0206031F0338032A
:106800008800EA44E944E244040005000600070069
:10681000080009000A000B000C000D000E000F001C
:1068200010001100120013001400150016001700CC
:10683000180019001A001B001C001D001E001F007C
:10684000200021002200230024002500260027002C
:10685000280029002A002B002C002D002E002F00DC
:10686000300031003200330034003500360037008C
:10687000380039003A003B003C003D003E003F003C
:1068800040004100420043004400450046004700EC
:10689000480049004A004B004C004D004E004F009C
:1068A000500051005200530054005500560057004C
:1068B000580059005A005B005C005D005E005F00FC
:1068C00060006100620063006400F1A18500670060
:1068D000680069006A006B006C006D006E006F005C
:1068E0007000710072007300890087008A008B00BD
:1068F000E000E100E200E300E400E500E600E7007C
:106900000100010001000100EA4401000100E2442D
:106910000100010001000100460001004A004B0097
:10692000010001004700480001000100E9440100A6
:106930000100010001000100010001003A003B00DC
:106940003C003D003E003F0040004100420043004B
:10695000010035004C0001000100440045005200D8
:1069600049000100010050004F0029004D004E0079
:1069700051000100010001000100010001000100BF
:1069800001000100010001000100010001000100FF
:1069900001000100010001000100010001004D00A3
:1069A0004A004E004B0001000100010001000100FF
:1069B00001000100010001000100010001000100CF
:1069C00001000100010001000100010001000100BF
:1069D00001000100010001000100010001000100AF
:1069E0000100010001000100490001000100010057
:1069F000010001000100010001000100010001008F
:00000001FF
